:100000000EC013C012C011C010C00FC00EC00DC072
:100010000CC00BC00AC009C008C007C006C011242C
:100020001FBECFEDCDBF22D06BC0EACF20ED37E0B1
:1000300003C0F9013197F1F70197D8F70895369A7F
:100040003699FECF85B1089582E088BD85E090E0C5
:10005000EDDF18BC88EC90E0E9CF8AE088BD84E64B
:1000600090E0E4DF18BC88EC90E0E0CF82E087BB52
:1000700081E28ABD81E083BF81EA87B9A29A86ECDA
:1000800086B9479A8FEF88BD85E090E0CFDF18BC36
:10009000D6DF18BC18E0C0E0D0E0D1DFC80FD11D1A
:1000A00082E390E0C3DF1150C1F783E0D695C79596
:1000B0008A95E1F703C0C456D109CFDFC436D10514
:1000C000D0F788EE93E0B2DFCA30D10520F4BCDF70
:1000D00002C02A97C2DFCA30D105D8F788EE93E074
:1000E000A5DF209721F4B0DF02C02197B6DF20976B
:1000F000E1F788EE93E09ADF88EB9BE097DFC9CFCA
:04010000F894FFCFA1
:00000001FF
